:020000040000FA
:1000000054EF26F0120012000EEF00F01200010073
:10001000464D000000010000B2000000DACFE4FF0E
:10002000E2CFDAFFE9CFE4FFEACFE4FFF6CFE4FF67
:10003000F7CFE4FFF5CFE4FFF3CFE4FFF4CFE4FF25
:10004000FACFE4FF00EE18F0140EE80403E3EECF5D
:10005000E4FFFBD700EE00F0180EE80403E3EECF58
:10006000E4FFFBD7E6529EAA3BD0B0EC25F00F018F
:100070002B6FABA40BD0AB9E3681342B000E3523F7
:10008000AB8EB0EC25F00F012B6F2B6BABA20AD01F
:10009000AB983683AB88B0EC25F00F012B6F322B79
:1000A000000E33230D0E2B5D0EE0000E1325E96EBE
:1000B000080E1421EA6E2BCFEFFF132B000E142332
:1000C0002C6B2D6B0CD0000E1325E96E080E14213D
:1000D000EA6EEF6A010E2C6F2D6B136B146B9E9AF8
:1000E0009EA018D00F012E2B000E2F23100E2E5D78
:1000F000000E2F5906E32E6B2F6B3685302B000E2A
:100100003123DB0EE66E0B0EE66ECFEC25F0E552EA
:10011000E5529E90E55200EE17F0180EE80403E356
:10012000E5CFEDFFFBD700EE2BF0140EE80403E360
:10013000E5CFEDFFFBD7E5CFFAFFE5CFF4FFE5CF45
:10014000F3FFE5CFF5FFE5CFF7FFE5CFF6FFE5CF0E
:10015000EAFFE5CFE9FFE5CFDAFF1100D9CFE6FFEF
:10016000E1CFD9FFFF0EE76EFD0EDBCF00F0FE0EF4
:10017000DBCF01F0E7500016016A0050A96EFD0EBA
:10018000DBCF00F0FE0EDBCF01F001C000F0016A12
:10019000030E0014AA6EA69EA69CA680A85000D0AE
:1001A000E552E7CFD9FF1200D9CFE6FFE1CFD9FF63
:1001B000020EE126DE6ADD6AFD0EDBCF00F0FE0EE8
:1001C000DBCF01F001C000F0016A030E0014AA6E3B
:1001D000FF0EE76EFD0EDBCF00F0FE0EDBCF01F071
:1001E000E7500016016A0050A96EFC0EDB50A86EA5
:1001F000A69EA684A69CF2AE04D0F29E010EDE6EF0
:10020000DD6A550EA76EAA0EA76EA682A1A8FED71C
:10021000A198A694D9CFE9FFDACFEAFF010EEE1834
:1002200001E1ED5001E1F28E020EE15C02E2E16AD1
:10023000E552E16EE552E7CFD9FF1200D9CFE6FFD4
:10024000E1CFD9FFFB0EDBCFE9FFFC0EDBCFEAFFEE
:10025000EF501DE0FB0EDBCFE9FFDB2AFC0EDBCF0E
:10026000EAFF01E3DB2AEF50E66EFD0EDBCF00F084
:10027000DB2AFE0EDBCF01F001E3DB2A00C0E6FF44
:1002800001C0E6FF91DFE552E552E552DBD7E552CA
:10029000E7CFD9FF1200D9CFE6FFE1CFD9FF030E98
:1002A000E126010EDB6A020EF36EF3CFDBFFFD0EDB
:1002B000DBCF00F0FE0EDBCF01F0013404E2005092
:1002C0000008000E015418E2140EE76E010EDBCF99
:1002D00000F0020EDBCF01F0E7500026000E0122F5
:1002E000010E00C0DBFF020E01C0DBFFFD0EDB06CE
:1002F000FE0E01E2DB06DBD70F01006B016B140E73
:10030000005D000E01591CE2010EDB5000250001CA
:10031000006E020EDB500F0101210001016E00C0D2
:10032000E6FF01C0E6FF1ADFE552E552DF6EDFCFE0
:10033000E6FF11DAE5520F01002B000E0123DFD793
:10034000030EE15C02E2E16AE552E16EE552E7CFBD
:10035000D9FF1200D9CFE6FFE1CFD9FFE652D9503D
:10036000FD0FE96EFF0EDA20EA6EFF0ED880EE5424
:10037000030EED5401E21BD0FD0EDBCFE6FFFE0EB7
:10038000DBCFE6FFEBDEE552E552DF6EDF5001E149
:100390000ED0DFCFE6FFE66AB3EC0EF0E552E55291
:1003A000FD0EDB2AFE0E01E3DB2ADF50D8E1E80E6A
:1003B000E66E030EE66EE66AE66AD0EC0EF0E552F3
:1003C000E552E552E552E552E552E7CFD9FF12007A
:1003D000D9CFE6FFE1CFD9FF040EE126200EDE6E75
:1003E000A10EDE6E070EDE6EDD6ADD52DD52D9CF64
:1003F000E9FFDACFEAFFD880000EEE54000EEE548B
:10040000000EEE54000EEE540AE2D9CFE9FFDACF27
:10041000EAFFEE06000EEE5AEE5AEE5AE8D7040E48
:10042000E15C02E2E16AE552E16EE552E7CFD9FF15
:100430001200D9CFE6FFE1CFD9FF020EE126DE6A36
:10044000DD6A0801005119E1DECF00F0DDCF01F0D7
:10045000880E005C130E015810E20A0EE66EE66A82
:10046000E66AE66AD0EC0EF0E552E552E552E55256
:10047000DF2A010E01E3DB2AE4D7DECF00F0DDCF77
:1004800001F0026AD8900250000A06E6500E005CA5
:10049000C30E0158000E025808E3C50EE66E450E65
:1004A000E66E19DAE552E55229D0960EE66E04ECB6
:1004B00026F0E55208010051000817E2000E0F0176
:1004C0001325E96E080E1421EA6EEF6A000EE66E3F
:1004D000080EE66E3CDAE552E5520F012C6B2D6BEF
:1004E0002B6B136B146B0801006BDECF00F0DDCFBC
:1004F00001F000C0F3FF01C0F4FF00D0020EE15C88
:1005000002E2E16AE552E16EE552E7CFD9FF12005F
:10051000010EE66EE66EC9D8E552E552010EE66EB2
:10052000020EE66EC2D8E552E552C20EE66E450EE8
:10053000E66E3FEC0EF0E552E552F3CF06FFF4CF46
:1005400007FF010EE66E800EE66EAFD8E552E5526B
:10055000BD0EE66E450EE66EBED9E552E55269DF88
:10056000F3CF1AFFF4CF1BFF640EE66E04EC26F007
:10057000E552AF0EE66E450EE66E3FEC0EF0E5522C
:10058000E552F3CF06FFF4CF07FF010EE66EC00E73
:10059000E66E8BD8E552E552A80EE66E450EE66E85
:1005A0009AD9E552E55245DFF3CF1AFFF4CF1BFF8E
:1005B000640EE66E04EC26F0E5529D0EE66E450EE6
:1005C000E66E3FEC0EF0E552E552F3CF06FFF4CFB6
:1005D00007FF010EE66E940EE66E67D8E552E5520F
:1005E000970EE66E450EE66E76D9E552E55221DFAE
:1005F000F3CF1AFFF4CF1BFF640EE66E04EC26F077
:10060000E5528E0EE66E450EE66E3FEC0EF0E552BC
:10061000E552F3CF06FFF4CF07FF010EE66ED40ECE
:10062000E66E43D8E552E552870EE66E450EE66E5D
:1006300052D9E552E552FDDEF3CF1AFFF4CF1BFF8E
:10064000E80EE66E04EC26F0E5521200D9CFE6FF84
:10065000E1CFD9FF020EE126C580C5B0FED7FE0E60
:10066000DBCFE6FFDBEC24F0E552DF6EFF0EDF5C54
:1006700004E1010EC9CFDBFFC69EFD0EDBCFE6FF16
:10068000DBEC24F0E552DF6EC584C5B4FED7DF5045
:10069000006E020EE15C03E200D0E16AE552E16E19
:1006A0000050E552E7CFD9FF1200D9CFE6FFE1CFE6
:1006B000D9FFE6520F01106BFE0EDB50F00B08095C
:1006C000DF6E040EDF10E66E0ECFE6FFBFDFE552F1
:1006D000E5520F01106F010EE66E7EEC26F0E5523A
:1006E000FB0EDF14E66E0ECFE6FFB0DFE552E552FB
:1006F0000F01106F010EE66E7EEC26F0E552FD0E46
:10070000DB5024E0FE0EDB38F00BF00B0809DF6E47
:10071000040EDF10E66E0ECFE6FF98DFE552E552DD
:100720000F01106F020EE66E7EEC26F0E552FB0E16
:10073000DF14E66E0ECFE6FF89DFE552E5520F01CA
:10074000106F010EE66E7EEC26F0E552E552E552A2
:10075000E7CFD9FF1200D9CFE6FFE1CFD9FFE652AC
:10076000FE0EDB50F00B08090109DF6E040EDF10EE
:10077000E66E0ECFE6FF6ADFE552E5520F01106F1D
:10078000020EE66E7EEC26F0E552FB0EDF14E66EFE
:100790000ECFE6FF5BDFE552E5520F01106F010E51
:1007A000E66E7EEC26F0E552FE0EDB38F00BF00B29
:1007B00008090109DF6E040EDF10E66E0ECFE6FFBA
:1007C00045DFE552E5520F01106F010EE66E7EEC3B
:1007D00026F0E552FB0EDF14E66E0ECFE6FF36DFA5
:1007E000E552E5520F01106F010EE66E7EEC26F029
:1007F000E552E552E552E7CFD9FF1200F40EE66E5E
:1008000004EC26F0E552E66A300EE66E4EDFE55265
:10081000E552640EE66E04EC26F0E552E66A300E10
:10082000E66E43DFE552E5520A0EE66E04EC26F072
:10083000E552E66A300EE66E38DFE552E552050E07
:10084000E66E04EC26F0E552E66A200EE66E2DDF39
:10085000E552E552050EE66E04EC26F0E552010E77
:10086000E66E280EE66E21DFE552E552050EE66ED5
:1008700004EC26F0E552010EE66E080EE66E15DF7A
:10088000E552E552050EE66E04EC26F0E552010E47
:10089000E66EE66E0ADFE552E552050EE66E04EC02
:1008A00026F0E552010EE66E060EE66EFEDEE5521D
:1008B000E552050EE66E04EC26F0E552010EE66EFA
:1008C0000C0EE66EF2DEE552E552140EE66E04EC16
:1008D00026F0E5521200D9CFE6FFE1CFD9FF020E94
:1008E000E126DE6ADD6AFD0EDBCFF6FFFE0EDBCF12
:1008F000F7FF0800F55021E0DECF00F0DDCF01F07A
:10090000D890015004E6140E005C000E015815E268
:10091000FD0EDBCFF6FFFE0EDBCFF7FF0800F55034
:10092000E66E19DFE552FD0EDB2AFE0E01E3DB2A3F
:10093000DF2A010E01E3DB2AD6D7020EE15C02E2D8
:10094000E16AE552E16EE552E7CFD9FF1200D9CF57
:10095000E6FFE1CFD9FF020EE126DE6ADD6AFD0E79
:10096000DBCFE9FFFE0EDBCFEAFFEF5020E0DECF6A
:1009700000F0DDCF01F0D890015004E6140E005CC9
:10098000000E015814E2FD0EDBCFE9FFFE0EDBCFB7
:10099000EAFFEF50E66EDFDEE552FD0EDB2AFE0ECB
:1009A00001E3DB2ADF2A010E01E3DB2AD8D7020E9E
:1009B000E15C02E2E16AE552E16EE552E7CFD9FF80
:1009C0001200D9CFE6FFE1CFD9FF020EE126FD0EDE
:1009D000DBCF1EF0FE0EDBCF1FF0040E1E1801E170
:1009E0001F5031E0030E1E1801E11F5021E0020EDE
:1009F0001E1801E11F5011E0010E1E1801E11F50E9
:100A000001E02CD0800EDE6EDD6A010EE66E800EF7
:100A1000E66E4BDEE552E55221D0C00EDE6EDD6A99
:100A2000010EE66EC00EE66E40DEE552E55216D0CF
:100A3000940EDE6EDD6A010EE66E940EE66E35DE15
:100A4000E552E5520BD0D40EDE6EDD6A010EE66E85
:100A5000D40EE66E2ADEE552E55200D0020EE66EB6
:100A600004EC26F0E552000EE66EE66A14DCE55270
:100A7000E552020EE66E04EC26F0E552010EE66E3B
:100A8000DFCFE6FF12DEE552E552020EE15C02E244
:100A9000E16AE552E16EE552E7CFD9FF120037D89F
:100AA000C580C5B0FED7120032D8C582C5B2FED708
:100AB00012002DD8C584C5B4FED71200D9CFE6FFE9
:100AC000E1CFD9FF9E96FE0EDB50C96E9EA6FED7E3
:100AD000E552E7CFD9FF1200D9CFE6FFE1CFD9FF2A
:100AE00016D8C586C5B6FED7C7A0FED7FE0EDBCF8B
:100AF000E6FF19D8E552C95000D0E552E7CFD9FF3B
:100B00001200280EC66E180EC86E9E961200640E55
:100B1000E66EE66AE66AE66AD0EC0EF0E552E55269
:100B2000E552E5521200D9CFE6FFE1CFD9FFFE0E24
:100B3000DB5002E0C58A01D0C59AC588C5B8FED78A
:100B4000E552E7CFD9FF1200D9CFE6FFE1CFD9FFB9
:100B50000A0E026E02C024F0FE0EDBCF1FF070EC16
:100B600026F01BC001F00A0E006E00C024F0FE0E3D
:100B7000DBCF1FF070EC26F01F38F00B011000D017
:100B8000E552E7CFD9FF1200D9CFE6FFE1CFD9FF79
:100B9000FE0EDB380F0B070B0A0DF3CF00F0FE0E35
:100BA000DB500F0B002400D0E552E7CFD9FF120035
:100BB000D9CFE6FFE1CFD9FFFC0EDB9EFD0EDB9E19
:100BC000FE0EDB9E6CDFD00EE66E78DFE552E66A45
:100BD00075DFE552FC0EDBCFE6FFB6DFE552E66ED1
:100BE0006DDFE552FD0EDBCFE6FFAEDFE552E66ED0
:100BF00065DFE552FE0EDBCFE6FFA6DFE552E66ECF
:100C00005DDFE55256DFE552E7CFD9FF120047DF3F
:100C1000D00EE66E53DFE552E66A50DFE55244DF60
:100C2000D10EE66E4BDFE552E66A56DFE552E66E20
:100C3000ABDFE5520901B26FE66A4EDFE552E66EC0
:100C4000A3DFE5520901B16F010EE66E45DFE55203
:100C5000E66E9ADFE5520901B06F59EF05F0D9CF82
:100C6000E6FFE1CFD9FF1BDFD00EE66E27DFE552AE
:100C7000030EE66E23DFE552FB0EDBCFE6FF64DFFB
:100C8000E552E66E1BDFE552FE0EDBCFE6FF5CDFD2
:100C9000E552E66E13DFE552FD0EDBCFE6FF54DFD3
:100CA000E552E66E0BDFE552FC0EDBCFE6FF4CDFD4
:100CB000E552E66E03DFE552100EE66EFFDEE5520A
:100CC000F8DEE552E7CFD9FF1200E9DED00EE66E7E
:100CD000F5DEE552030EE66EF1DEE552E5DED10EFD
:100CE000E66EECDEE552E66AF7DEE552E66E4CDFD4
:100CF000E5520901B36FE66AEFDEE552E66E44DFC6
:100D0000E5520901B66FE66AE7DEE552E66E3CDFC2
:100D1000E5520901B46F010EE66EDEDEE552E66EC5
:100D200033DFE5520901B56F59EF05F0D9CFE6FF82
:100D3000E1CFD9FF0901B26BF90EDBCFB1F9FA0EA1
:100D4000DBCFB0F9FB0EDBCFB3F9FC0EDBCFB6F98E
:100D5000FD0EDBCFB4F9FE0EDBCFB5F9A0DED00E71
:100D6000E66EACDEE552E66AA9DEE552B2C9E6FF00
:100D7000EBDEE552E66EA2DEE552B1C9E6FFE4DE47
:100D8000E552E66E9BDEE552B0C9E6FFDDDEE552D8
:100D9000E66E94DEE552B3C9E6FFD6DEE552E66EB6
:100DA0008DDEE552B6C9E6FFCFDEE552E66E86DEA1
:100DB000E552B4C9E6FFC8DEE552E66E7FDEE552D5
:100DC000B5C9E6FFC1DEE552E66E78DEE552100EEB
:100DD000E66E74DEE5526DDEE552E7CFD9FF120014
:100DE000D9CFE6FFE1CFD9FF040EE126020EDE6E79
:100DF000DD6A0F01026B036B9D9A000EE66E080E12
:100E0000E66E66EC24F0E552E552020EF3CFDBFF0E
:100E1000030EF4CFDBFF020EDBCFE9FF030EDBCFC7
:100E2000EAFFE906000EEA5A000EE926080EEA2259
:100E3000EF50E66EE66A08010051E66EE66A000EC3
:100E4000E66E080EE66E020EDBCFE6FF030EDBCF8A
:100E5000E6FF440E006E450E016E026A00C0E6FF1A
:100E600001C0E6FF02C0E6FFFE0EE66EE668FFEC9C
:100E700023F0036E0D0EE15E0350F3CF04FFF4CFB9
:100E800005FF550E0801005D01E0DFD0020EDBCF4B
:100E9000E9FF030EDBCFEAFFE906000EEA5A000E77
:100EA000E926080EEA22EF50230801E0CED0020E18
:100EB000DBCF00F0030EDBCF01F0D890015004E649
:100EC000150E005C000E015801E3BFD0020EDBCF0F
:100ED000E6FF030EDBCFE6FF000EE66E080EE66EC1
:100EE000210E006E450E016E026A00C0E6FF01C0D1
:100EF000E6FF02C0E6FFFE0EE66EE668FFEC23F0BA
:100F0000036E090EE15E0350F3CF04FFF4CF05FF3B
:100F1000020E0F01006F016B020EDBCF00F0030E1B
:100F2000DBCF01F00050005D015001593DE2000EA1
:100F30000025E96E080E0121EA6EEF503B0830E112
:100F4000000E0025E96E080E0121EA6EEF6ADECF81
:100F500000F0DDCF01F0000E0026080E012200C0D7
:100F6000E6FF01C0E6FF7BEC1FF0E552E552F350CF
:100F7000E66EB70E0F010225E96E090E0321EA6E37
:100F8000E552E750EF6E010E016A0025006E015137
:100F9000012200C0DEFF01C0DDFF022B000E032393
:100FA000002B000E0123B8D7020EDBCFE9FF030EA2
:100FB000DBCFEAFFE906000EEA5A000EE926080E2A
:100FC000EA22EF6ADECF00F0DDCF01F0000E00264E
:100FD000080E012200C0E6FF01C0E6FF7BEC1FF017
:100FE000E552E552F350E66EB70E0F010225E96EA9
:100FF000090E0321EA6EE552E750EF6EBCC9B1F964
:10100000BBC9B0F9B7C9B6F9B8C9B4F9B9C9B5F926
:10101000BAC9B3F9B1C9E6FFB0C9E6FFB3C9E6FF83
:10102000B6C9E6FFB4C9E6FFB5C9E6FF7FDE006ECC
:10103000060EE15E00500801006B0F01026B036BAE
:101040002C6B2D6B136B146B9D8A040EE15C02E21A
:10105000E16AE552E16EE552E7CFD9FF1200D9CF40
:10106000E6FFE1CFD9FF0E0EE126F90EDBCFDEFF62
:10107000DBCFDDFFF80EDBCF02F0000EE76E0218CB
:10108000E8AE02D0023403D0E750D880025402E325
:10109000070E12D0F80EDBCF03F0160EE76E031822
:1010A000E8AE02D0033403D0E750D880035402E204
:1010B000170E02D0F80EDB28006E016A00BE016830
:1010C000080E00C0DBFF090E01C0DBFF020EDB6A69
:1010D000030EDB6AFB0EDBCF00F0FC0EDBCF01F072
:1010E000FD0EDBCF02F0FE0EDBCF03F0226A236A97
:1010F000246A256A00C01DF001C01EF002C01FF066
:1011000003C020F06AEC1EF0010A33E1F90EDBCFD8
:10111000E9FFDB2AFA0EDBCFEAFF01E3DB2A2D0E23
:10112000EF6EFB0EDBCF00F0FC0EDBCF01F0FD0E0F
:10113000DBCF02F0FE0EDBCF03F0226A236A800EC3
:10114000246EBF0E256E00C01DF001C01EF002C04F
:101150001FF003C020F08EEC1DF0FB0E1DC0DBFF66
:10116000FC0E1EC0DBFFFD0E1FC0DBFFFE0E20C00D
:10117000DBFFFB0EDBCF00F0FC0EDBCF01F0FD0E42
:10118000DBCF02F0FE0EDBCF03F0226A236A246A73
:10119000256A00C01DF001C01EF002C01FF003C090
:1011A00020F061EC1EF0010A4AE1FB0EDBCF00F0FB
:1011B000FC0EDBCF01F0FD0EDBCF02F0FE0EDBCF2D
:1011C00003F0226A236A800E246E3F0E256E00C053
:1011D0001DF001C01EF002C01FF003C020F06AEC39
:1011E0001EF0010A2CE1006A016A200E026E410E17
:1011F000036ED950FB0FE96EFF0EDA20EA6EEECFD8
:101200001DF0EECF1EF0EECF1FF0EFCF20F000C0AC
:1012100022F001C023F002C024F003C025F08EECC0
:101220001DF020C0EDFF1FC0EDFF1EC0EDFF1DC073
:10123000EFFF020EDB06030E01E2DB06B6D7FB0E64
:10124000DBCF00F0FC0EDBCF01F0FD0EDBCF02F0B8
:10125000FE0EDBCF03F0226A236A200E246E410EBD
:10126000256E00C01DF001C01EF002C01FF003C0BB
:1012700020F06AEC1EF0010A2EE0FB0EDBCF00F03E
:10128000FC0EDBCF01F0FD0EDBCF02F0FE0EDBCF5C
:1012900003F0226A236A200E246E410E256E00C0E0
:1012A0001DF001C01EF002C01FF003C020F03BEC97
:1012B0001DF0FB0E1DC0DBFFFC0E1EC0DBFFFD0E94
:1012C0001FC0DBFFFE0E20C0DBFF020EDB2A030E79
:1012D00001E3DB2AB4D7020EDBCF00F0030EDBCF35
:1012E00001F0D950080FE96EDACFEAFF0050EE2680
:1012F0000150ED22010EF36E040EF3CFDBFF050E5D
:10130000DB6A040EDBCF1EF0050EDBCF1FF076ECA0
:101310001CF00A0E1DC0DBFF0B0E1EC0DBFF0C0E07
:101320001FC0DBFF0D0E20C0DBFF040EDBCF00F083
:10133000050EDBCF01F0080EDBCF02F0090EDBCF8C
:1013400003F001500318E8AE02D0033404D0025079
:10135000005C035001582EE20A0EDBCF00F00B0EAA
:10136000DBCF01F00C0EDBCF02F00D0EDBCF03F074
:10137000226A236A200E246E410E256E00C01DF0E5
:1013800001C01EF002C01FF003C020F03BEC1DF0B6
:101390000A0E1DC0DBFF0B0E1EC0DBFF0C0E1FC0B4
:1013A000DBFF0D0E20C0DBFF040EDB2A050E01E380
:1013B000DB2ABBD70A0EDBCF04F00B0EDBCF05F028
:1013C0000C0EDBCF06F00D0EDBCF07F0226A236A8E
:1013D000246A400E256E04C01DF005C01EF006C034
:1013E0001FF007C020F03BEC1DF01DC000F01EC038
:1013F00001F01FC002F020C003F0D950FB0FE96ECE
:10140000FF0EDA20EA6EEECF1DF0EECF1EF0EECF2B
:101410001FF0EFCF20F000C022F001C023F002C087
:1014200024F003C025F0A5EC1CF020C0EDFF1FC088
:10143000EDFF1EC0EDFF1DC0EFFFFB0EDBCF00F088
:10144000FC0EDBCF01F0FD0EDBCF02F0FE0EDBCF9A
:1014500003F0226A236A200E246E410E256E00C01E
:101460001DF001C01EF002C01FF003C020F06AECA6
:101470001EF0010A13E0FB0EDB6AFC0EDB6A800E35
:10148000F36EFD0EF3CFDBFF3F0EF36EFE0EF3CFD8
:10149000DBFF020EDB2A030E01E3DB2A020EDBCFA9
:1014A00000F0030EDBCF01F00001800E01145FE0BD
:1014B000F90EDBCFE9FFDB2AFA0EDBCFEAFF01E30F
:1014C000DB2A300EEF6EF90EDBCFE9FFDB2AFA0ED6
:1014D000DBCFEAFF01E3DB2A2E0EEF6E080EDBCF37
:1014E00000F0090EDBCF01F0800E011414E0020EB3
:1014F000DBCF02F0030EDBCF03F0080EDB50025C03
:10150000006E090EDB500358016E020E00C0DBFFB7
:10151000030E01C0DBFF040EDB68050EDB68040E62
:10152000DBCF00F0050EDBCF01F0020EDBCF02F0C7
:10153000030EDBCF03F003500118E8AE02D00134F4
:1015400004D00050025C0150035811E2F90EDBCFC9
:10155000E9FFDB2AFA0EDBCFEAFF01E3DB2A300EDC
:10156000EF6E040EDB06050E01E2DB06D8D7040E93
:10157000DB6A050EDB6A040EDBCF00F0050EDBCF65
:1015800001F0080EDBCF02F0090EDBCF03F00150B3
:101590000318E8AE02D0033404D00250005C0350BC
:1015A000015801E3ACD0FB0EDBCF1DF0FC0EDBCF0E
:1015B0001EF0FD0EDBCF1FF0FE0EDBCF20F0FBECAC
:1015C0001DF0060E1EC0DBFF070E1FC0DBFF300E36
:1015D000E76E060EDBCF00F0070EDBCF01F0E75021
:1015E0000026000E0122F90EDBCFE9FFDB2AFA0EFE
:1015F000DBCFEAFF01E3DB2A00C0EFFF040EDBCF05
:1016000000F0050EDBCF01F0020EDB50001803E105
:10161000030EDB5001180BE1F90EDBCFE9FFDB2AEB
:10162000FA0EDBCFEAFF01E3DB2A2E0EEF6E060E89
:10163000DBCF1EF0070EDBCF1FF076EC1CF00A0E9E
:101640001DC0DBFF0B0E1EC0DBFF0C0E1FC0DBFF3F
:101650000D0E20C0DBFF1DC000F01EC001F01FC03A
:1016600002F020C003F0D950FB0FE96EFF0EDA2024
:10167000EA6EEECF1DF0EECF1EF0EECF1FF0EFCFF3
:1016800020F000C022F001C023F002C024F003C00B
:1016900025F0A4EC1CF020C0EDFF1FC0EDFF1EC024
:1016A000EDFF1DC0EFFF006A016A200E026E410EC1
:1016B000036ED950FB0FE96EFF0EDA20EA6EEECF13
:1016C0001DF0EECF1EF0EECF1FF0EFCF20F000C0E8
:1016D00022F001C023F002C024F003C025F08EECFC
:1016E0001DF020C0EDFF1FC0EDFF1EC0EDFF1DC0AF
:1016F000EFFF040EDB2A050E01E3DB2A3CD7F90ECF
:10170000DBCFE9FFFA0EDBCFEAFFEF6A0E0EE15CFA
:1017100002E2E16AE552E16EE552E7CFD9FF12003D
:10172000D9CFE6FFE1CFD9FF060EE1260F01369DA6
:10173000FB0EDBCF1DF0FC0EDBCF1EF0FD0EDBCF72
:101740001FF0FE0EDBCF20F02AEC1EF01CC0DEFFE7
:101750001DC0DEFF1EC0DEFF1FC0DDFFDD52DD52FB
:10176000FB0EDBCF04F0FC0EDBCF05F0FD0EDBCF74
:1017700006F0FE0EDBCF07F0F90EDBCF1EF0FA0EFF
:10178000DBCF1FF076EC1CF01DC008F01EC009F086
:101790001FC00AF020C00BF008C022F009C023F0DF
:1017A0000AC024F00BC025F004C01DF005C01EF0D7
:1017B00006C01FF007C020F08EEC1DF01DC000F029
:1017C0001EC001F01FC002F020C003F0F90EDBCFF5
:1017D00014F0FA0EDBCF15F0166A176A15AE02D0B8
:1017E0001668176814C01CF015C01DF016C01EF056
:1017F00017C01FF0DFCF21F0010EDBCF22F0020E69
:10180000DBCF23F0030EDBCF24F054EC25F018C01F
:1018100010F019C011F01AC012F01BC013F010C064
:101820001CF011C01DF012C01EF013C01FF08BEC95
:101830001CF01DC00CF01EC00DF01FC00EF020C02B
:101840000FF00CC022F00DC023F00EC024F00FC02A
:1018500025F000C01DF001C01EF002C01FF003C043
:1018600020F0A4EC1CF0FBEC1DF0040E1EC0DBFF0E
:10187000050E1FC0DBFF800EE66E080EE66ED9CFA8
:10188000E9FFDACFEAFFEECFE6FFEECFE6FFEECFDD
:10189000E6FFEFCFE6FF5FEC21F0006E060EE15EA3
:1018A0000050800EE66E080EE66E24DAE552E55230
:1018B000F3CF04FFF4CF05FF2E0EE66EE66A53DA8F
:1018C000E552E552E66A040EDBCFE6FF050EDBCFFC
:1018D000E6FF0DD8E552E552E552060EE15C02E264
:1018E000E16AE552E16EE552E7CFD9FF1200D9CFA8
:1018F000E6FFE1CFD9FF0A0EE1260F012D0E206F82
:10190000010E216FFC0EDBCF00F0010EE76E001818
:10191000E8AE02D0003403D0E750D880005401E292
:10192000DBD0FC0EDB5028E1FD0EDBCF00F0FE0E1D
:10193000DBCF01F0060E00C0DBFF070E01C0DBFFAE
:10194000080EDB6A090EDB6A2D0EE66E010EE66EEE
:10195000D950060FE96EDACFEAFFEECFE6FFEECF01
:10196000E6FFEECFE6FFEFCFE6FF5FEC21F0006E83
:10197000060EE15E005010D02D0EE66E010EE66EF2
:10198000FD0EDBCFE6FFFE0EDBCFE6FFF0EC1FF037
:10199000E552E552E552E5520F0136AD84D02D0EE9
:1019A000E66E010EE66E66EC24F0E552E552020E9C
:1019B000F3CFDBFF030EF4CFDBFFDE6ADD6ADECFA1
:1019C00000F0DDCF01F0020EDBCF02F0030EDBCF23
:1019D00003F00250005C035001582EE2020EDBCFF0
:1019E00002F0030EDBCF03F0DE50025CE96EDD5047
:1019F0000358EA6EE906000EEA5A2D0EE926010E9A
:101A0000EA22EF50E66EFC0EDB50040F006E016A16
:101A100000BE0168DE50005CE96EDD500158EA6EE0
:101A20002D0EE926010EEA22E552E750EF6EDF2A7D
:101A3000010E01E3DB2AC3D7DE6ADD6ADECF00F0E8
:101A4000DDCF01F0FC0EDB50050F046E056A04BE0D
:101A50000568020EDB50045C026E030EDB50055875
:101A6000036E0250005C035001581DE20F0136A9BD
:101A70000BD0DECFE9FFDDCFEAFF2D0EE926010E08
:101A8000EA22300EEF6E0AD0DECFE9FFDDCFEAFFAB
:101A90002D0EE926010EEA22200EEF6EDF2A010E3E
:101AA00001E3DB2ACBD7FC0EDB50050FE96EEA6AB7
:101AB000E9BEEA682D0EE926010EEA22EF6A20CF80
:101AC000E6FF21CFE6FF16D9E552E552020EF3CF2D
:101AD000DBFF030EF4CFDBFF0A0EE15C02E2E16AFA
:101AE000E552E16EE552E7CFD9FF1200D9CFE6FF0C
:101AF000E1CFD9FFE652800EDF6EDF50000821E211
:101B0000DF50F36EFE0EDBCFF4FFF350F45C0FE317
:101B1000310EE66EE66A27D9E552E552FE0EDB503D
:101B2000D880DF54E76EFE0EE7CFDBFF06D0300E25
:101B3000E66EE66A18D9E552E552DF407F0BDF6EAC
:101B4000DCD7E552E552E7CFD9FF1200D9CFE6FF47
:101B5000E1CFD9FF020EE126FE0EDB50F00BE83894
:101B60000F0B300FDF6EDF50390803E2070EDF2462
:101B7000DF6EFE0EDB500F0B300FE76E010EE7CF6E
:101B8000DBFFDB5039080AE2070E006E010EDBCFE7
:101B9000E7FF0050E726010EE7CFDBFFDFCFE6FFD0
:101BA000E66AE1D8E552E552010EDBCFE6FFE66AD0
:101BB000DAD8E552E552680EE66EE66AD4D8E55208
:101BC000E552020EE15C02E2E16AE552E16EE552A5
:101BD000E7CFD9FF12000101005107E1C20E011940
:101BE00004E1010E021901E1035130E0005106E168
:101BF000960E011903E1025101E1035122E0005167
:101C000006E14B0E011903E1025101E1035114E019
:101C1000800E001906E1250E011903E1025101E1D0
:101C2000035105E0820E0F01116F126B14D0820E6A
:101C30000F01116F126B0FD0400E0F01116F126B5D
:101C40000AD0200E0F01116F126B05D00A0E0F0182
:101C5000116F126B00D0410E116F126B11CFE6FFA6
:101C600012CFE6FF740EE66E1BEC25F0E552E5524E
:101C7000E5529F8AD08E9D9AF29CF29E1200D9CF97
:101C8000E6FFE1CFD9FF020EE126DE6ADD6AFD0E36
:101C9000DBCFF6FFFE0EDBCFF7FF0800F55017E0B5
:101CA000FD0EDBCFF6FFFE0EDBCFF7FF0800F55091
:101CB000E66EE66A58D8E552E552DF2A010E01E3E6
:101CC000DB2AFD0EDB2AFE0E01E3DB2AE0D7DECFA6
:101CD00000F0DDCF01F000C0F3FF01C0F4FF020E01
:101CE000E15C03E200D0E16AE552E16EE552E7CF44
:101CF000D9FF1200D9CFE6FFE1CFD9FF020EE126CE
:101D0000DE6ADD6AFD0EDBCFE9FFFE0EDBCFEAFF08
:101D1000EF5016E0FD0EDBCFE9FFFE0EDBCFEAFF52
:101D2000EF50E66EE66A1FD8E552E552DF2A010E53
:101D300001E3DB2AFD0EDB2AFE0E01E3DB2AE2D7FC
:101D4000DECF00F0DDCF01F000C0F3FF01C0F4FFF3
:101D5000020EE15C03E200D0E16AE552E16EE55279
:101D6000E7CFD9FF1200D9CFE6FFE1CFD9FFACA270
:101D7000FED7FD0EDBCFE6FF1BEC26F0E552E55269
:101D8000E7CFD9FF12000D0EE66EE66AECDFE552F2
:101D9000E5520A0EE66EE66AE6DFE552E55212000B
:101DA000D9CFE6FFE1CFD9FFFB0EDBCF1DF0FC0E54
:101DB000DBCF1EF0FD0EDBCF1FF0FE0EDBCF20F0E1
:101DC0002034000E201809E6D880000E1D54000EA5
:101DD0001E54000E1F54000E20540CE2D950FB0F6D
:101DE000E96EFF0EDA20EA6EEE06000EEE5AEE5AAB
:101DF000EE5ADAD7E552E7CFD9FF12000F013F8F35
:101E00003F9D3F8B3F893F873F853F833F913E8F7B
:101E10003E9D3E893E873E853E833E813D873D8592
:101E20003D833D918168396B93689380938293845D
:101E300093869388938A938C938EF19E6168386B16
:101E40003881388338852F0E926E82683A6BBF0EC8
:101E5000946E949C948ED08ED09C606A1200CD9E1D
:101E6000CD9CCD8ACD88CD96CD94CD82CD90CC9E83
:101E7000CC9ACC92CC909F80D08EDB0EE66E0B0E6F
:101E8000E66ECFEC25F0E552E5529E90F29CCD90A7
:101E90009D90F29EF29C1200D9CFE6FFE1CFD9FFD0
:101EA000020EE126FD0EDBCFDEFFDBCFDDFFDECF56
:101EB00000F0DDCF01F0D89000360136D890003622
:101EC00001360050C26EC280050EE66E7EEC26F032
:101ED000E552A0EC26F09BEC26F0000901E0FBD7D0
:101EE00089EC26F0F3CF0AFFF4CF0BFF0F0136B7D2
:101EF00032D04D0EE66EE66A36DFE552E552310E1F
:101F0000E76EFD0EDBCF00F0FE0EDBCF01F0E750F9
:101F10000026000E012200C0E6FF01C0E6FF23DF1D
:101F2000E552E5523D0EE66EE66A1DDFE552E552EA
:101F30000F01368DE66A0ACFE6FF0BCFE6FFD7DC4E
:101F4000E552E552E5520F01369D3B0EE66EE66A1C
:101F50000ADFE552E552020EE15C02E2E16AE55277
:101F6000E16EE552E7CFD9FF120048DF0F01368D51
:101F7000368936953697346B356B326B336B89887F
:101F80002C6B2D6B0801006B0F01369F24DE9EAA7F
:101F900005D0B0EC25F00F012B6FF9D70F012B6B9B
:101FA0000C0EE66EE66ADFDEE552E552A00EE66E46
:101FB000860EE66E010EE66EE66AF2DEE552E55248
:101FC000E552E552000EE66EE66AAAEC01F0E55233
:101FD000E552200EE66EE66AAAEC01F0E552E55203
:101FE000400EE66EE66AAAEC01F0E552E552600E9C
:101FF000E66EE66AAAEC01F0E552E552800EE66E66
:10200000E66AAAEC01F0E552E552A00EE66EE66A39
:10201000AAEC01F0E552E552E66A010EE66EAAEC82
:1020200001F0E552E552200EE66E010EE66EAAECD6
:1020300001F0E552E552E66A030EE66EAAEC01F005
:10204000E552E5520101800E3E6F080E3F6F06C15A
:1020500000F007C101F0026A00C0E6FF01C0E6FF20
:1020600002C0E6FF3EC1E6FF3FC1E6FF4DEC24F0B3
:10207000036E050EE15E035000C11CFF01C11DFF90
:1020800002C11EFF03C11FFF0A0E0101016A3E25A6
:10209000006E3F51012200C0E6FF01C0E6FF1CCFE9
:1020A000E6FF1DCFE6FF1ECFE6FF1FCFE6FF8AEC5F
:1020B00020F0026E060EE15E02503EC1E6FF3FC117
:1020C000E6FF66EC24F0E552E552F3CF00FFF4CFD3
:1020D00001FF01013E510F010025E96E01013F5151
:1020E0000F010121EA6E2E0EEF6E3EC1E6FF3FC1E9
:1020F000E6FF00DEE552E552F3CF04FFF4CF05FF23
:1021000008C1E6FF09C1E6FFBADDE552E552F3CFAB
:1021100006FFF4CF07FF0EC1E6FF0FC1E6FFAFDDFC
:10212000E552E552F3CF06FFF4CF07FF2CDEF00EA9
:10213000E66E490EE66E020EE66EE66A31DEE552A6
:10214000E552E552E552C69A0F014E0E0E6F800E13
:10215000E66E080EE66EEBEC25F0E552E552180E41
:10216000C86EC750040B01E0010E006E1F0EC514AF
:10217000001001E0F6D7C580C5B0FED7C9CF0FFF6C
:102180000ECFE6FFDBEC24F0E5520F01106FFF0EDF
:10219000105D03E1C9CF0FFFC69E022B000E032383
:1021A000105105E0640E025D000E0359E9E3640E70
:1021B000025D000E035920E202CFE6FF03CFE6FFE7
:1021C0000E51E66EE66AF70E006E440E016E026A6C
:1021D00000C0E6FF01C0E6FF02C0E6FFFE0EE66EAD
:1021E000E668FFEC23F0036E090EE15E0350F3CFC7
:1021F00004FFF4CF05FF22D002CFE6FF03CFE6FFB6
:102200001051E66EE66A0E51E66EE66ABD0E006E8D
:10221000440E016E026A00C0E6FF01C0E6FF02C084
:10222000E6FFFE0EE66EE668FFEC23F0036E0B0E93
:10223000E15E0350F3CF04FFF4CF05FFA4DD0F01EF
:102240004E0E0E6FFEEC03F00F01106B010EE66EEA
:10225000E66E55EC03F0E552E552010EE66E020E15
:10226000E66E55EC03F0E552E5520F014E0E0E6F8F
:10227000FEEC03F0100EE66E270EE66EE66AE66AE6
:102280008FDDE552E552E552E552010EE66EE66E4F
:1022900055EC03F0E552E552010EE66E020EE66ED5
:1022A00055EC03F0E552E552010EE66E800EE66E47
:1022B00055EC03F0E552E552010EE66EE66A4BEC92
:1022C00001F0E552E552010EE66EC00EE66E55ECE9
:1022D00003F0E552E552020EE66EE66A4BEC01F0C1
:1022E000E552E552010EE66E940EE66E55EC03F0F3
:1022F000E552E552030EE66EE66A4BEC01F0E5525C
:10230000E552010EE66ED40EE66E55EC03F0E55292
:10231000E552040EE66EE66A4BEC01F0E552E5523A
:10232000800EE66E1A0EE66E060EE66EE66A38DD82
:10233000E552E552E552E55280BA12D0060EE66E3D
:10234000100EE66E050EE66E170EE66E080EE66ED1
:102350000D0EE66E96EC06F0006E060EE15E005085
:1023600007EC06F0030EE66EE66AE1EC04F0E552D7
:10237000E5520901B251E66EE66AB151E66EE66ACF
:10238000B051E66EE66AA30E006E440E016E026A5C
:1023900000C0E6FF01C0E6FF02C0E6FF3EC1E6FF67
:1023A0003FC1E6FF5AEC23F0036E0B0EE15E0350D3
:1023B000F3CF04FFF4CF05FF3EC1E6FF3FC1E6FFC8
:1023C000A7EC04F0E552E552E80EE66E030EE66E69
:1023D000E66AE66AE5DCE552E552E552E55265EC6F
:1023E00006F0040EE66EE66AE1EC04F0E552E55212
:1023F0000901B551E66EE66AB451E66EE66AB65179
:10240000E66EE66A890E006E440E016E026A00C036
:10241000E6FF01C0E6FF02C0E6FF3EC1E6FF3FC1A6
:10242000E6FF5AEC23F0036E0B0EE15E0350F3CF90
:1024300004FFF4CF05FF3EC1E6FF3FC1E6FFA7EC76
:1024400004F0E552E552800EE66E1A0EE66E060EB8
:10245000E66EE66AA5DCE552E552E552E5520F016B
:10246000369F2B6B136B146B326B336B346B356B8A
:1024700036913693AB889D8AF28CF28E2C6B2D6B45
:102480002B6B0801006B0F01136B146B353504E2E5
:1024900034510008000E355507E3333504E232515C
:1024A0000008000E335536E204C1E6FF05C1E6FF21
:1024B0003FEC0EF0E552E552F3CF06FFF4CF07FFF5
:1024C000090EE66EE66A4FDCE552E552E66A34CF65
:1024D000E6FF35CFE6FF77EC0CF0E552E552E5522A
:1024E000090EE66EE66A3FDCE552E552E66A32CF57
:1024F000E6FF33CFE6FF77EC0CF0E552E552E5520C
:1025000042DC0F012B6B0801006B0F01136B146B86
:102510002C6B2D6B100EE66E270EE66EE66AE66AF1
:102520003FDCE552E552E552E552020EE66EE66A00
:10253000E1EC04F0E552E552030EE66EE66AE1ECEA
:1025400004F0E552E552040EE66EE66AE1EC04F0B2
:10255000E552E552010EE66E800EE66E55EC03F094
:10256000E552E5520F01136B146B2B6B0801006BE6
:102570000F012C6B2D6B88EC02F0C280C19EC08EC7
:10258000C08AC088C096C094C082C090C196C194D1
:10259000C192C1900F013697898861DC9E90F28CC0
:1025A000F28EF28C9D80CD800F013695086B096B01
:1025B0002E6B2F6B2B6B306B316B030EE66EE66A66
:1025C000E1EC04F0E552E552040EE66EE66AE1EC59
:1025D00004F0E552E5520801300E006F010E0F01C4
:1025E0002C6F2D6B3687369508014C0E006F020E4E
:1025F0000F01136F146B0F013651040B03E12C51C3
:102600002D11F9E0010EE66E800EE66E55EC03F03A
:10261000E552E55207EC06F00901B251E66EE66AB2
:10262000B151E66EE66AB051E66EE66A700E006E73
:10263000440E016E026A00C0E6FF01C0E6FF02C060
:10264000E6FF3EC1E6FF3FC1E6FF5AEC23F0036E12
:102650000B0EE15E0350F3CF04FFF4CF05FF3EC144
:10266000E6FF3FC1E6FFA7EC04F0E552E552530E4A
:10267000E66EE66AB3EC0EF0E552E5523D0EE66E0C
:10268000E66AB3EC0EF0E552E55281CF15FF15CFA7
:10269000E6FF76EC0DF0E5523B0EE66EE66AB3EC33
:1026A0000EF0E552E552010EE66EC00EE66E55ECF8
:1026B00003F0E552E5520F013651080B01E0010E1F
:1026C000E66EE66A1551E66EE66A5D0E006E440E31
:1026D000016E026A00C0E6FF01C0E6FF02C0E6FF2D
:1026E0003EC1E6FF3FC1E6FF5AEC23F0036E090E40
:1026F000E15E0350F3CF04FFF4CF05FF3EC1E6FFD8
:102700003FC1E6FFA7EC04F0E552E5520F01010ED0
:102710002C1901E12D5101E08ED1080100514C0A24
:1027200001E15AD1190A01E12CD1660A01E1F5D083
:10273000010A01E1BED0030A01E187D0740A5BE01F
:10274000040A2FE0130A29E0010EE66EE66AE1ECC6
:1027500004F0E552E552FC0E006E430E016E026A73
:1027600000C0E6FF01C0E6FF02C0E6FF3EC1E6FF93
:102770003FC1E6FF5AEC23F0036E050EE15E035005
:10278000F3CF04FFF4CF05FF3EC1E6FF3FC1E6FFF4
:10279000A7EC04F0E552E55222D10F01086B096B5A
:1027A0001ED18998010EE66EE66AE1EC04F0E5526E
:1027B000E5524D0E006E440E016E026A00C0E6FF47
:1027C00001C0E6FF02C0E6FF3EC1E6FF3FC1E6FFF3
:1027D0005AEC23F0036E050EE15E0350F3CF04FFC5
:1027E000F4CF05FF3EC1E6FF3FC1E6FFA7EC04F0D2
:1027F000E552E552F4D08988010EE66EE66AE1EC16
:1028000004F0E552E5523D0E006E440E016E026A80
:1028100000C0E6FF01C0E6FF02C0E6FF3EC1E6FFE2
:102820003FC1E6FF5AEC23F0036E050EE15E035054
:10283000F3CF04FFF4CF05FF3EC1E6FF3FC1E6FF43
:10284000A7EC04F0E552E552CAD0000EE66EE66A47
:102850004CEC0FF0E552E552030EE66EE66AE1EC51
:1028600004F0E552E5520ACFE6FF0BCFE6FF320E49
:10287000006E440E016E026A00C0E6FF01C0E6FF72
:1028800002C0E6FF3EC1E6FF3FC1E6FF5AEC23F07F
:10289000036E070EE15E0350F3CF04FFF4CF05FF94
:1028A0003EC1E6FF3FC1E6FFA7EC04F0E552E5526A
:1028B00096D0010EE66EE66A4CEC0FF0E552E5525A
:1028C000030EE66EE66AE1EC04F0E552E5520ACF4B
:1028D000E6FF0BCFE6FF270E006E440E016E026A84
:1028E00000C0E6FF01C0E6FF02C0E6FF3EC1E6FF12
:1028F0003FC1E6FF5AEC23F0036E070EE15E035082
:10290000F3CF04FFF4CF05FF3EC1E6FF3FC1E6FF72
:10291000A7EC04F0E552E55262D0020EE66EE66ADC
:102920004CEC0FF0E552E552030EE66EE66AE1EC80
:1029300004F0E552E5520ACFE6FF0BCFE6FF1C0E8E
:10294000006E440E016E026A00C0E6FF01C0E6FFA1
:1029500002C0E6FF3EC1E6FF3FC1E6FF5AEC23F0AE
:10296000036E070EE15E0350F3CF04FFF4CF05FFC3
:102970003EC1E6FF3FC1E6FFA7EC04F0E552E55299
:102980002ED0010EE66EE66AE1EC04F0E552E55267
:102990000C0E006E440E016E026A00C0E6FF01C01C
:1029A000E6FF02C0E6FF3EC1E6FF3FC1E6FF5AEC8C
:1029B00023F0036E050EE15E0350F3CF04FFF4CF66
:1029C00005FF3EC1E6FF3FC1E6FFA7EC04F0E5527C
:1029D000E552F0EC06F003D00F01367700D0040E7C
:1029E000E66EE66AE1EC04F0E552E55208010051BA
:1029F000E66EE66AE80E006E430E016E026A00C0E3
:102A0000E6FF01C0E6FF02C0E6FF3EC1E6FF3FC1B0
:102A1000E6FF5AEC23F0036E070EE15E0350F3CF9E
:102A200004FFF4CF05FF3EC1E6FF3FC1E6FFA7EC80
:102A300004F0E552E5520F0136A7A1D0030EE66E71
:102A4000E66AE1EC04F0E552E552E20E006E430E58
:102A5000016E026A00C0E6FF01C0E6FF02C0E6FFA9
:102A60003EC1E6FF3FC1E6FF5AEC23F0036E050EC0
:102A7000E15E0350F3CF04FFF4CF05FF3EC1E6FF54
:102A80003FC1E6FFA7EC04F0E552E5520F01026BEF
:102A9000036B030E025D000E035970E202CFE6FFE6
:102AA00003CFE6FF4CEC0FF0E552E5524D0EE66E1B
:102AB000E66AB3EC0EF0E552E552310E0F01016A01
:102AC0000225006E0351012200C0E6FF01C0E6FFAF
:102AD000B3EC0EF0E552E5523D0EE66EE66AB3EC5D
:102AE0000EF0E552E5520F01368DE66A0ACFE6FF99
:102AF0000BCFE6FF77EC0CF0E552E552E5520F0103
:102B0000369D3B0EE66EE66AB3EC0EF0E552E552FA
:102B10000ACFE6FF0BCFE6FFDC0E006E430E016E20
:102B2000026A00C0E6FF01C0E6FF02C0E6FF3EC148
:102B3000E6FF3FC1E6FF5AEC23F0036E070EE15EAD
:102B40000350F3CF04FFF4CF05FF3EC1E6FF3FC1C2
:102B5000E6FFA7EC04F0E552E552E80EE66E030E40
:102B6000E66EE66AE66AD0EC0EF0E552E552E55212
:102B7000E5520F01022B000E03238BD732D04C0EEF
:102B80000801005D2EE10F013651080B2AE1030E0A
:102B9000E66EE66AE1EC04F0E552E552C80E006E1E
:102BA000430E016E026A00C0E6FF01C0E6FF02C0EC
:102BB000E6FF3EC1E6FF3FC1E6FF5AEC23F0036E9D
:102BC000050EE15E0350F3CF04FFF4CF05FF3EC1D5
:102BD000E6FF3FC1E6FFA7EC04F0E552E55208012D
:102BE000006B08010051000804E20F01086B096B3B
:102BF00004D00F01082B000E0923000ED8800855C1
:102C0000000E095551E208CF00F009CF01F0000194
:102C1000016A0F0E00160050011046E1C3EC0EF0E1
:102C20000CC1E6FF0DC1E6FF3FEC0EF0E552E552A8
:102C3000F3CF06FFF4CF07FFE66A08CFE6FF09CF20
:102C4000E6FF77EC0CF0E552E552E552200EE66E19
:102C5000E66AB3EC0EF0E552E55212C1E6FF13C18D
:102C6000E6FF3FEC0EF0E552E552F3CF06FFF4CF5E
:102C700007FFF40EE66E010EE66EE66AE66AD0EC39
:102C80000EF0E552E552E552E552040EE66EE66AB4
:102C9000E1EC04F0E552E55212C1E6FF13C1E6FF94
:102CA0006BEC04F0E552E5520F0136A503D03695E2
:102CB0002E6B2F6B2B6B2C6B2D6B0801006BC3ECF9
:102CC0000EF099D412009FEC1BF0FB0EDBCFF3FF4C
:102CD000DB06F35000090AE0EDEC1BF0FA0E58ECAD
:102CE0001CF0F3E1011CF1E1010E01D0000ECEEF6A
:102CF0001BF09FEC1BF03B0EE12402E3E168E6527F
:102D0000E16E010EDB6A020EDB6AF90EDBCFF6FF25
:102D1000FA0EDBCFF7FFFB0EDBCFF8FF0800F55014
:102D2000DF6EDF5002E1F2EF1AF0250EDF5C02E009
:102D3000E5EF1AF0030EDB6A040EDB6A050EDB6AB0
:102D4000060EDB6A070EDB6A07EC1BF02D0EDF5C5C
:102D50000CE02B0EDF5C09E0200EDF5C06E0230EAA
:102D6000DF5C03E0300EDF5C1AE1DF50300A14E074
:102D7000130A0FE0030A0AE00B0A05E0060AE4E181
:102D8000030EDB80E1D7030EDB82DED7030EDB848C
:102D9000DBD7030EDB86D8D7030EDB88D5D72A0E08
:102DA000DF5C1BE103EC1BF051EC1BF010E0030EA9
:102DB000DB801E681F68130EDBCF23F0140EDBCF01
:102DC00024F04EEC1FF0040E1CC0DBFF03D0130EEA
:102DD0003AEC1BF007EC1BF00BD0090EDB6AA8ECF9
:102DE0001BF003E01CEC1CF0FAD7090E3AEC1BF0C8
:102DF000030EDBB0DB982E0EDF5C1BE107EC1BF053
:102E00002A0EDF5C0BE103EC1BF051EC1BF003E13D
:102E1000130E8CEC1BF007EC1BF00BD0090EDB6AD9
:102E2000A8EC1BF003E01CEC1CF0FAD7090E8CECAC
:102E30001BF0680EDF5C07E107EC1BF0680EDF5C3F
:102E40001DE1030E18D0740EDF5C17E07A0EDF5C14
:102E500014E0480EDF5C06E0540EDF5C03E05A0E1F
:102E6000DF5C02E1020E07D06C0EDF5C03E06A0E4D
:102E7000DF5C04E1010EDFEC1BF0C9DBDF506E0A02
:102E800001E17FD31E0A01E192D1200A01E18FD135
:102E90003F0A01E149D11A0A01E146D10D0A01E1D7
:102EA00043D1200A01E140D13A0A01E13DD1200A93
:102EB00001E13AD1260A01E135D10D0A01E132D111
:102EC0001A0A01E1D9D0200A4AE0300A1FE0460A76
:102ED0000EE0250A01E083D3D950F90FE96EFF0E09
:102EE000DA20EA6E010EEE5E000EEE5AEE5AEDECBE
:102EF0001BF0250EE66E95DB03E1011C01E169D3B1
:102F0000E9EC1BF001E26BD3DB2A69D3080EDB6A24
:102F1000040EDB50010806E2040EDB04B1EC1BF0EA
:102F2000DB508BDB080EDB5009E0030EDB50010B9E
:102F300005E172DB01E04DD3080EDB6A64DBEFCF05
:102F4000DFFF61EC1CF003E1011C01E142D3E9EC7D
:102F50001BF001E3DB2A60DB01E141D33AD3070E2A
:102F6000DB5002080FE12DEC1CF0030EF4EC1BF01B
:102F70000E0EEECFDBFF0F0EEECFDBFF100EEECF0F
:102F8000DBFF20D0F70EDBCF03F0F80EDBCF04F031
:102F9000020E035E000E045AF70E03C0DBFFF80EAC
:102FA00004C0DBFF03C0E9FF04C0EAFFE4EC1BF050
:102FB000026A0E0E00C0DBFF0F0E01C0DBFF100E19
:102FC00002C0DBFF0E0EDBCFE6FF0F0EDBCFE6FF0E
:102FD000100EDBCFE6FF74EC24F0E552E552E5522B
:102FE000130E1DC0DBFF140E1EC0DBFF060EDB50F0
:102FF00005E0130E28EC1CF001E26ADB4CEC1CF03F
:1030000002E2130E37DB0FEC1CF006E0040E28EC96
:103010001CF002E2050E2EDB030EDBB005D0FCDA5D
:1030200001E0D7D2080EDB6A090EDB6A0E0EDBCF99
:10303000F6FF0F0EDBCFF7FF100EDBCFF8FF080017
:10304000F550DF6EDF5014E052EC1CF011E261EC41
:103050001CF003E1011C01E1BCD2BBDB01E3DB2A74
:10306000090EDB2AD9500E0FE96E000ECBDBE7D735
:10307000D3DA01E1B4D2ADD2C6DA110EEECFDBFF66
:10308000120EEDCFDBFF110EDBCFE6FF120EDBCF12
:10309000E6FF66EC24F0E552E552130EF3CFDBFFBA
:1030A000140EF4CFDBFF060EDB5004E0130ED0DB72
:1030B00001E20EDB4CEC1CF002E2130EDBDAAFDBBC
:1030C00005E0040EC5DB02E2050ED4DA030EDBB028
:1030D00005D0A2DA01E07DD2080EDB6A090EDB6AB8
:1030E000110EDBCFE9FF120EDBCFEAFFEFCFDFFFE0
:1030F000DF5014E0D7DB12E2E4DB03E1011C01E165
:1031000068D267DB01E3DB2A090EDB2A110EDB2A1A
:10311000DBCFE9FF120EE8E3DB2AE6D77DDA01E137
:103120005ED257D2030EDB8E070EDB0410E195DB77
:10313000040E5ADB0A0EEECFDBFF0B0EEECFDBFFE9
:103140000C0EEECFDBFF0D0EEECFDBFF6CD0070ECB
:10315000DB5003082CE1030EDBAE0DD0B2DA020E19
:1031600076DAEFCF00F0016A026A036A00AE39D066
:103170000168026835D0F70EDBCF01F0F80EDBCF27
:1031800002F0020E015E000E025AF70E01C0DBFFD4
:10319000F80E02C0DBFF01C0E9FF02C0EAFFEFCF7B
:1031A00000F00A0E00C0DBFF0B0EDB6A38D0070E02
:1031B000DB50020809E1030EDBAE04D059DB02AE9E
:1031C00010D00ED055DB0DD0030EDBAE12D079DA65
:1031D000020E3DDAF9DA026A036A01AE02D0026831
:1031E0000368E2DA0C0E02C0DBFF0D0E03C0DBFF4A
:1031F0001AD0F70EDBCF02F0F80EDBCF03F0020E91
:10320000025E000E035AF70E02C0DBFFF80E03C089
:10321000DBFF02C0E9FF03C0EAFFD6DAC5DA0C0E15
:10322000DB6A0D0EDB6A060EDB5005E1010EF36E64
:10323000050EF3CFDBFF150EDB6A160EDB6AD950E5
:10324000370F006E000EDA20016E390E00C0DBFF72
:103250003A0E01C0DBFF380EDB6A080EDB6A0A0E8D
:10326000AEDADF50780A12E0200A10E0280A0CE0FB
:10327000200A0AE03F0A06E00D0A02E0200A08E1FF
:10328000020E05D0080E03D0080EDF26100E97DAC6
:10329000030EDBBE02D0DB92DB94DB50800B24E01C
:1032A0008ADAD890030EEB50000A08E6000EEE5CB6
:1032B000000EEE58000EEE58000EEE5815E213DA2E
:1032C000216822682368246854EC25F00A0E18C08F
:1032D000DBFF0B0E19C0DBFF0C0E1AC0DBFF0D0E5F
:1032E0001BC0DBFF2D0E08D0030EDBA202D02B0E7D
:1032F00003D0DBA408D0200EF36E170EF3CFDBFF54
:10330000150EDB2A02D0170EDB6A050EDB5003E137
:10331000B7D901E189D0240E006E4D0E016E000E6A
:10332000026E070EDBCF03F0046A056A066A03C06B
:1033300021F004C022F005C023F006C024F0D3D948
:103340008CEC25F000501824F36E01501920F46E17
:1033500002501A20F86EF4CFF7FFF3CFF6FF080003
:10336000090EF5CFDBFF580EDF5C0FE1610EF36E47
:10337000090E7BD90AE3200E006E090EDBCFE7FFB2
:103380000050E75E090EE7CFDBFF070EDBCF00F052
:10339000016A026A036A0FDA00C021F001C022F05C
:1033A00002C023F003C024F0EECF1CF0EECF1DF0DE
:1033B000EECF1EF0EFCF1FF08CEC25F01FC0EDFF1D
:1033C0001EC0EDFF1DC0EDFF1CC0EFFF390EDBCFAF
:1033D000E9FFDB063A0EDBCFEAFF01E2DB06090E6E
:1033E000DBCFEFFF150EDB2A4BD995E1030EDBA6F1
:1033F0001DD06F0EDF5C06E1C1D918E3150EDB2886
:103400005BDA14D0780EDF5C09E0580EDF5C06E072
:10341000620EDF5C03E0420EDF5C08E1020EF36E39
:10342000160EF3CFDBFF02D0150EDB6A030EDB5066
:10343000100B0EE0040EDBCF00F0050EDB50D88041
:10344000005406E2060EDB5003E1040EDB5034DAD2
:1034500095D90AE2050EDBCFE7FF150EDB50E75EDC
:10346000050EE7CFDBFF02D0050EDB6A040EDBCFD3
:1034700000F0160E45D9D880005414E2160EDBCFAA
:10348000E6FF150EDBCFE6FF040EDBCFE6FF050EF1
:10349000DB50E552E75CE552D880E754E552D8802E
:1034A000E7545FD9030EDB50010B0BE1080EDB5034
:1034B00008E0B2D801E08DD0080EDB50BED8080E6F
:1034C000DB6A170EDB5007E088D9170EF1D903E14C
:1034D000011C01E17ED0160EDB5016E07ED9300EC5
:1034E000E66E9FD802E1011C74E077D9DFCFE6FFDA
:1034F00099EC24F0E552E552E552F4CF01F00001D9
:10350000F31C02E1011C65E0050EDBCF00F0160E96
:10351000DB50D880005409E2050EDBCFE7FF160E22
:10352000DB50E75E050EE7CFDBFF300EE66E050EE3
:10353000CBD94FE1390EDB2ADBCFE9FF3A0E01E3AD
:10354000DB2ADBCFEAFF090EEFCFDBFFDB500EE01B
:1035500044D9090EADD902E1011C3BE0390EDB2A4A
:10356000DBCFE9FF3A0EEDE3DB2AEBD755D831E1AB
:10357000160EDBCFE6FF080EC3D8E552E7245DD870
:103580002ED0070EDB50030A1CE0010A14E0030AE8
:1035900007E07BD9DBCFEEFF020EDBCFEDFF1FD0C4
:1035A000F5D8056A03AE02D0046805682CD8BCD8EB
:1035B00005C0EEFF14D0EAD803BE046824D8B4D8FE
:1035C0000ED063D9DBCFEFFF0AD07BD905E1011C18
:1035D00003E1F368F46810D0FCD801E3DB2A79D961
:1035E0008EEF16F0010EDBCF00F0020EDBCF01F004
:1035F00000C0F3FF01C0F4FF3B0EE15C02E2E16AB0
:10360000E552E16ECBD029D9020EF4EF1BF061D95F
:103610000800F550DF6E1200200EE66E080E64EF13
:103620001CF099EC24F0E552E552E552F3CF00F09E
:10363000F4CF01F00001F31C1200006E016AD950B2
:10364000010F4DD90050EE260150ED221200045E0C
:10365000000E055AF70E04C0DBFFF80E05C0DBFFB5
:1036600004C0E9FF05C0EAFF1200DBCFF4FFF3500E
:10367000F45C1200DB50E76E040EE7CFDBFF1200B4
:103680000A0EDBCF00F00B0EDBCF01F00C0EDBCF10
:1036900002F00D0EDBCF03F00050011002100310FA
:1036A0001200130EEECFDBFF140EEDCFDBFF130E77
:1036B000DBCF00F0140EDBCF01F00001800E01140F
:1036C0001200F70EDBCF04F0F80EDBCF05F012008E
:1036D000050EDB50E66ED950130F01D9E552E750C5
:1036E000EE6EED6A12000A0EDBCF1CF00B0EDBCF84
:1036F0001DF00C0EDBCF1EF00D0EDBCF1FF0120005
:10370000DBCFE6FF150EDBCFE6FF050EDB50E55203
:10371000E724E552E7241200DB50CED8010EF36E09
:10372000060EF3CFDBFF1200EE50EFCFEAFFE96E9B
:1037300002C0EEFF03C0EEFF04C0EEFF1200D9CFBF
:10374000E6FFDACFE6FFE1CFD9FFE2CFDAFF1200E2
:10375000DFCFE6FFE66A32EC26F0E552E552F350A1
:103760001200E76E080EE7CFDBFF1200EECF00F08D
:10377000EECF01F0EFCF02F0036A1200050EDBCFAF
:1037800000F0150EDB50D88000541200010EDBCF84
:1037900002F0020EDBCF03F0046A1200E552E5CF1F
:1037A000DAFFE7CFD9FF12000A0E00C0DBFF0B0ED5
:1037B00001C0DBFF1200D9500A0F6FEF1CF0F36E4F
:1037C000070EF3CFDBFF1200EECF00F0EFCF01F0DA
:1037D0001200010EDB2A020E1200FC0EDBCFE6FF08
:1037E000FD0EDBCFE6FF1200005E000E015AF70E61
:1037F00000C0DBFFF80E01C0DBFF00C0E9FF01C025
:10380000EAFF1200DA20EA6EEF2AEECFF6FF000E92
:10381000EF22EECFF7FFEF22EECFF8FF1200040EFB
:10382000DBCFE6FF130EDB50E552E75C9ADFDB509F
:1038300004DF060EDB501200090EDB500A0DF350B8
:10384000DF24D00FE76E090EE7CFDBFF07EF1BF099
:10385000DB50F36E050E35EF1BF0F70EDBCF00F0FB
:10386000F80EDBCF01F01200DFCFE6FF11EF1BF007
:1038700028DF030EECDEB6EF1BF063EC16F0E5522A
:10388000E552E552E55200091200BDDEEE50EFCFE1
:10389000EAFFE96E010E1200130EDB50F36E040E08
:1038A00035EF1BF0040EDB50F36E090E35EF1BF005
:1038B000DBCFE6FF11EF1BF0E76E050EE7CFDBFF76
:1038C00012008BDF34EF1CF0DBCFE6FF86DF3DEF2D
:1038D0001CF0D950F90FE96EFF0E02EF1CF0E96EF3
:1038E000000EDA20EA6E1200279E08D0279E1FAE37
:1038F00005D01E6C1F1EE86A1F22278E1FC019F0FC
:103900001EC018F02B6A2A6A8E0E1A6E1B6AE4EF2C
:103910001EF0279E0CD0279E1FAE09D01C6C1D1ECA
:103920001E1E1F1EE86A1D221E221F22278E1FC078
:1039300019F01EC018F01DC02BF01CC02AF09E0EFE
:103940001A6E1B6AE4EF1EF0257E276A20EC1FF03A
:1039500038EC1FF027B6C8EF1EF027A20AD027AA1E
:1039600003D027BEC8EF1EF027A4D4EF1EF0D1EF7E
:103970001EF027AA05D027ACD4EF1EF0D1EF1EF021
:1039800027A00AD027A808D027BE04D027A402D099
:10399000DDEF1EF0E1EF1EF02A6A1B6A2550205C65
:1039A000296E10E31DC02BF01EC018F01FC019F0C7
:1039B00020C028F022C01DF023C01EF024C01FF03C
:1039C000273A09D022C02BF023C018F024C019F0E8
:1039D00025C028F0296C279E27BC278E28C01AF006
:1039E00027B010EF1FF01A0E296010EF1FF01A6AAF
:1039F000206A27A408D01D6C1E1E1F1E201EE86A08
:103A00001E221F22202227AC08D02B6C181E191E44
:103A10001A1EE86A182219221A221C6A295207E083
:103A200020341F321E321D321C32292EF9D71D5070
:103A30002B261E5018221F50192220501A221CC05B
:103A40002AF0279E1AAE0BD02A6C2B1E181E191EA8
:103A50001A1EE86A2B22182219221A22278E1AA06F
:103A600006D0D880193218322B322A32282A28C0A0
:103A70001AF0E4EF1EF0276A20EC1FF038EC1FF07C
:103A800027B6C8EF1EF027A205D027BAC8EF1EF050
:103A9000CFEF1EF027BADBEF1EF027A005D027B826
:103AA000C8EF1EF0DBEF1EF027B8CFEF1EF01B6A49
:103AB0007F0E20241A6EE86A1B2225501A5EE86ADF
:103AC0001B5A1A0E286E206A2A6A2B6A186A196A0B
:103AD00022501D5E23501E5A24501F5A000E205A99
:103AE00009E722501D2623501E2224501F22000EBB
:103AF000202201D02A8AD8901D361E361F36203645
:103B0000D8902A362B3618361936282EE1D71F5072
:103B10001E101D10D8A42A8AE4EF1EF0276A20EC9C
:103B20001FF038EC1FF027B6C8EF1EF027A205D013
:103B300027B8C8EF1EF0CFEF1EF027AA05D027B098
:103B4000C8EF1EF0CFEF1EF027B002D027A802D09A
:103B5000DBEF1EF01B6A255020241A6EE86A1B2238
:103B60007E0E1A5EE86A1B5A2A6A2B6A186A196A5C
:103B700024501F02F4CF19F0F3CF18F023501F0286
:103B8000F3502B26F4501822000E192224501E0246
:103B9000F3502B26F4501822000E192222501F0237
:103BA000F3502A26F4502B22000E182219222350FB
:103BB0001E02F3502A26F4502B22000E182219223E
:103BC00024501D02F3502A26F4502B22000E1822F6
:103BD000192222501E02F4502A26000E2B221822EF
:103BE000192223501D02F4502A26000E2B221822DF
:103BF0001922E4EF1EF0276A20EC1FF027B605EF2C
:103C00001EF027A20ED027B405D07F0E1F6EFF0E28
:103C10001E6E1FD0800E1F6E1E6A1BD01F6A1E6A8A
:103C200018D027B0FBD78F0E2060EDD77E0E206412
:103C3000F5D78E0E205C05E0D8901F321E32202A68
:103C4000F8D727A406D01E6C1F1EE86A1F221FAEDD
:103C5000E5D71200276A20EC1FF027B634EF1EF0DC
:103C600027A20FD027B407D07F0E1F6EFF0E1E6E47
:103C70001D6E1C6E25D0800E1F6E01D01F6A000EB7
:103C8000F6D727B0FBD71C6A9F0E2060EBD77E0EBD
:103C90002064F4D79E0E205C07E0D8901F321E32BD
:103CA0001D321C32202AF6D727A40AD01C6C1D1EF8
:103CB0001E1E1F1EE86A1D221E221F221FAEDED7F7
:103CC000120073EC1EF027B6000C27B0000C27B4CE
:103CD000000C010C73EC1EF027B6000C27B0000C92
:103CE00027A4000C010C276A20EC1FF038EC1FF011
:103CF00027B6120027AE08D027A004D027A802D0EC
:103D000027801200279012002550205C0BE12450E0
:103D10001F5C08E123501E5C05E122501D5C02E19E
:103D200027801200D8A002D0278E10D0205025C0A6
:103D300020F0256E1F5024C01FF0246E1E5023C09B
:103D40001EF0236E1D5022C01DF0226E2550205CF7
:103D500010E0FF0F09E0279027B403D027AE278497
:103D6000120027AE27941200252AD890243223323D
:103D7000223222501D5E23501E5A24501F5A1FBE4D
:103D8000EAD7D8901D361E361F36202EF8D7C8D752
:103D90007F0E206EFF0E1F6E1E6E1D6E12007F0EB8
:103DA00027BEFF0E206E02D07F0E206E800E1F6E8B
:103DB0001E6A1D6AF3D727AE04D0800E206E1F6ADC
:103DC000F7D7206A1F6AF4D7195018102B102A1041
:103DD000F8E01BBEF0D719BE0CD01A501B10EBE058
:103DE000D8902A362B36183619361A06D8A01B0654
:103DF000F2D71B50D4E11A28D2E02AAE11D07F0EA0
:103E00002A1402E12BA00CD02B2AE86A18221922CE
:103E100007E3D880193218322B321A2A1A28BFE049
:103E20001A50C9E02BC01DF018C01EF019341F6EC7
:103E30001A30206E1F32209E27BE208ECEEF1EF03D
:103E40001F36203602E32784277E06E12780206A7A
:103E50001F6A1E6A1D6A1200202803E0D8801F32E4
:103E60001200D8901F3202E127821200278612002A
:103E70002436253602E3278C277E06E12788256A2B
:103E8000246A236A226A1200252803E0D88024329B
:103E90001200D8902432EAE1278A12001FC02BF0CA
:103EA0001EC02AF01E502302F4CF1DF0F3CF1CF0E9
:103EB0001F502402F4CF1FF0F3CF1EF02302F35063
:103EC0001D26F4501E22E86A1F222A502402F350B5
:103ED0001D26F4501E22E86A1F2224AE74EF1FF044
:103EE0002A501E5E2B501F5A2BAE000C23501E5E14
:103EF00024501F5A000CFF0EE3CFEAFFE552FF0EDD
:103F0000E3CFE9FFE552E66AE66AD9CFE6FFDACF0A
:103F1000E6FFFC0EE124D96EFF0EE220DA6EE66ABF
:103F2000E66AE66A200EEF5C06E0090EEF5C03E04D
:103F3000EF6603D03FD0EE50F5D72D0EEF5C03E1D6
:103F4000FF0EE32A03D02B0EEF5C01E1EE502F0EA3
:103F5000EF6424D03A0EEF6021D0D890F90EE3360A
:103F6000FA0EE336FD0EDECFE3FFFE0EDDCFE3FFFC
:103F7000D890F90EE336FA0EE336D890F90EE33610
:103F8000FA0EE336FD0EE350DE26FE0EE350DD2290
:103F9000300EEE5CDE26000EDD22D9D7FF0EE3CF19
:103FA000E8FFE85207E0F90EE31EE32AFA0ED8B460
:103FB000E306E31EE552E552E552FF0EE3CFDAFFDA
:103FC000E552FF0EE3CFD9FFE552E1CFE9FFE2CFA3
:103FD000EAFFED52ED52EECFF3FFEFCFF4FF120008
:103FE000D9CFE6FFDACFE6FFFA0EE3CFD9FFFB0E1B
:103FF000E3CFDAFFFD0EE35209E72D0EDE6EFC0E75
:10400000E31EE32AFD0ED8B4E306E31EE652E652B1
:10401000E652FD0EE124E76EFF0EE220E46EE6526A
:10402000F70EE3CFE6FFF70EE3CFE6FF60EC20F0FC
:10403000F90EE124E96EFF0EE220EA6E50EC20F06A
:104040000AE14DEC20F009E150EC20F008E14DECE4
:1040500020F007E108D05BEC20F056EC20F05BECA0
:1040600020F056EC20F05BEC20F0DE6AF90EE12641
:10407000FF0EE222FF0EE3CFDAFFE552FF0EE3CFA1
:10408000D9FFE552FC0EE124E96EFF0EE220EA6E54
:10409000EECFF3FFEFCFF4FF1200EF380F0B12005B
:1040A000EF500F0B02E1EE52D8841200EF380F0BE5
:1040B000300FDE6E1200EE500F0B300FDE6E12006E
:1040C000FC0EE3CFE9FFFD0EE3CFEAFF100EE66E34
:1040D000EE6AEE6AEF6AD890FD0EE336FE0EE33626
:1040E000ED36ED36EF36FF0EE30609E081EC20F009
:1040F000EE5281EC20F0EE5281EC20F0EDD7E56E2F
:104100001200030EEF24E8B6EF6E300EEF24E8BE87
:10411000EF6E000CD9CFE6FFDACFE6FFF80EE3CF63
:10412000D9FFF90EE3CFDAFFFD0EE35215E72D0EAE
:10413000DE6EFA0EE31EFB0EE31EFC0EE31EFD0E0A
:10414000E31EFA0EE32A08E1FB0EE32A05E1FC0E6A
:10415000E32A02E1FD0EE32AE652E652E652E65277
:10416000E652FB0EE124E76EFF0EE220E46EE6521B
:10417000F30EE3CFE6FFF30EE3CFE6FFF30EE3CF5C
:10418000E6FFF30EE3CFE6FF27EC21F0F50EE12486
:10419000E96EFF0EE220EA6E14EC21F019E117EC53
:1041A00021F018E114EC21F017E117EC21F016E1F1
:1041B00014EC21F015E117EC21F014E114EC21F0DE
:1041C00013E117EC21F012E114EC21F011E112D00F
:1041D0001DEC21F022EC21F01DEC21F022EC21F06D
:1041E0001DEC21F022EC21F01DEC21F022EC21F05D
:1041F0001DEC21F022EC21F0DE6AF50EE126FF0E27
:10420000E222FF0EE3CFDAFFE552FF0EE3CFD9FF44
:10421000E552FA0EE124E96EFF0EE220EA6EEECFDF
:10422000F3FFEFCFF4FF1200EF380F0B1200EF5047
:104230000F0B02E1EE52D8841200EF380F0B300F53
:10424000DE6E1200EE500F0B300FDE6E1200FA0E13
:10425000E3CFE9FFFB0EE3CFEAFF200EE66EEE6A46
:10426000EE6AEE6AEE6AEF6AD890FB0EE336FC0E59
:10427000E336FD0EE336FE0EE336ED36ED36ED3673
:10428000ED36EF36FF0EE3060FE056EC21F0EE526E
:1042900056EC21F0EE5256EC21F0EE5256EC21F0A5
:1042A000EE5256EC21F0E1D7E56E1200030EEF243A
:1042B000E8B6EF6E300EEF24E8BEEF6E000CD9CFFB
:1042C000E6FFDACFE6FFF80EE3CFD9FFF90EE3CF32
:1042D000DAFFE652E652E652E652E652FB0EE124DF
:1042E000E76EFF0EE220E46EE652F30EE3CFE6FF48
:1042F000F30EE3CFE6FFF30EE3CFE6FFF30EE3CFDB
:10430000E6FF27EC21F0F50EE124E96EFF0EE22036
:10431000EA6ED1EC21F019E1D4EC21F018E1D1ECF6
:1043200021F017E1D4EC21F016E1D1EC21F015E1F8
:10433000D4EC21F014E1D1EC21F013E1D4EC21F024
:1043400012E1D1EC21F011E112D0DAEC21F0DFEC36
:1043500021F0DAEC21F0DFEC21F0DAEC21F0DFECF7
:1043600021F0DAEC21F0DFEC21F0DAEC21F0DFECE7
:1043700021F0DE6AF50EE126FF0EE222FF0EE3CF0A
:10438000DAFFE552FF0EE3CFD9FFE552FA0EE12442
:10439000E96EFF0EE220EA6EEECFF3FFEFCFF4FFFF
:1043A0001200EF380F0B1200EF500F0B02E1EE522C
:1043B000D8841200EF380F0B300FDE6E1200EE5073
:1043C0000F0B300FDE6E12004E6F20526571756557
:1043D000737420666F72204144432000253034649A
:1043E0002000414E413D20004C61737420436465C0
:1043F000203A202563202020202020004E6F2063BB
:104400006F6D7072656E646F20212000557064615D
:104410007465205254432064617461004144433305
:104420003D202530346400414443323D2025303462
:104430006400414443313D202530346400457465B7
:10444000696E74204C4544205241342000416C6C0C
:10445000756D65204C4544205241342000506F72E8
:1044600074423D20253038622054623D253162007F
:1044700054696D65206973202530326448253032D7
:10448000644D2530326453200044617465206973A3
:1044900020253032642F253032642F3230253032DF
:1044A00064200054696D65206973202530326448AA
:1044B000253032644D253032645320200050422094
:1044C00061647265737361676520253032582C20F2
:1044D000496E69742049324320494E636F72726598
:1044E000637465205374617475733D2533642020B3
:1044F0006A3D2535640D00496E6974205043463885
:1045000035373420636F727265637465204164725D
:10451000657373653D25303258206A3D2533640D3F
:10452000000A0D4D6973652061206C2768657572FE
:1045300065203A2025732020202532642063617293
:10454000730A0D000A0D4D6973652061206C2768A0
:10455000657572652064652025303364206361725F
:1045600073203D257320206275666665727B302955
:104570003D25632020204275666665725B6C2D3197
:104580005D3D25630A0D00424155443D20004154E4
:104590002B42415544340050494E3E200041542B9B
:1045A00050494E31323334004E414D453E2000419A
:1045B000542B4E414D456C696E766F720041543EEE
:1045C00020004154003F3F004672616D65204572F6
:1045D00072657572206574204F766572666C6F77B0
:1045E00020646574656374696F6E203A2000506FB3
:1045F000727420636F6D6D202E2E2E2E2E2E206253
:1046000064732C206F7576657274200D0A00313842
:104610004632364B32325F42545F59432D4D43553B
:104620005F4C43445F4453313330375F4331385F2D
:104630003133303832302E630D0A00455343207039
:104640006F757220736F727469720D004A3D20009D
:10465000496E697420425420466F72636565202854
:10466000656E2061766575676C65290D0A002020EE
:10467000202020202020202020202020202020203A
:104680002020004C696E6B2054696D656F75742035
:1046900045786365656420333220736563200D0AB5
:1046A000004461792000486F757220004D696E7575
:1046B00074652000D9CFE6FFDACFE6FFE1CFD9FF5E
:1046C000E2CFDAFFE652E652E652E652D950F90F4F
:1046D000006EFF0EDA20016E020E00C0DBFF030E3B
:1046E00001C0DBFF020EDBCFE6FF030EDBCFE6FFF0
:1046F000F90EDBCFE6FFFA0EDBCFE6FFFB0EDBCFDA
:10470000E6FFD950FC0FE66EFF0EDA20E66E79EC7C
:1047100016F0006E070EE15C02E2E16AE552E16E1E
:104720000050F3CFDEFFF4CFDDFFFC0EDBCFE9FF5F
:10473000FD0EDBCFEAFFEF6ADECF00F0DDCF01F048
:1047400000C0F3FF01C0F4FF040EE15C02E2E16A85
:10475000E552E16EE552E5CFDAFFE7CFD9FF12006F
:104760000E0EF66E000EF76E000EF86E01010900D7
:10477000F550B76F0900F550B86F03E1B76701D086
:104780003DD00900F550B26F0900F550B36F090034
:10479000F550B46F09000900F550E96E0900F550B5
:1047A000EA6E090009000900F550B56F0900F550DF
:1047B000B66F09000900F6CFB9F1F7CFBAF1F8CF1B
:1047C000BBF1B2C1F6FFB3C1F7FFB4C1F8FF0101FD
:1047D000B55302E1B65307E00900F550EE6EB50798
:1047E000F8E2B607F9D7B9C1F6FFBAC1F7FFBBC106
:1047F000F8FF0101B707000EB85BBFD71200D9CF91
:10480000E6FFDACFE6FFE1CFD9FFE2CFDAFFE652EB
:10481000E652E652E652D950F90F006EFF0EDA204A
:10482000016E00C0DEFFDD6EDECFE6FFDDCFE6FF0E
:10483000F90EDBCFE6FFFA0EDBCFE6FFFB0EDBCF98
:10484000E6FFFC0EDBCFE6FFFD0EDBCFE6FF79ECEB
:1048500016F0006E070EE15C02E2E16AE552E16EDD
:104860000050020EF3CFDBFF030EF4CFDBFF020E8E
:10487000DBCF00F0030EDBCF01F000C0F3FF01C07F
:10488000F4FF040EE15C02E2E16AE552E16EE552FA
:10489000E5CFDAFFE7CFD9FF1200FB0EE3CFF6FF3B
:1048A000FC0EE3CFF7FFFD0EE3CFF8FFFE0EE3CFE4
:1048B000E9FFFF0EE3CFEAFFE9CFF3FFEACFF4FF12
:1048C0000900F5CFEFFFEE66FBD71200FE0EE3CF37
:1048D000E9FFFF0EE3CFEAFFF36AF46AEE5203E06A
:1048E000F34AF42AFBD71200FF0EE3CFF8FFE5529C
:1048F000FF0EE3CFF7FFE552FF0EE3CFF6FFE552E1
:10490000E66AE66AE66A0900F55209E0FD0EE32A66
:1049100005E1FE0EE32A02E1FF0EE32AF4D7FD0EC5
:10492000E3CF1DF0FE0EE3CF1EF0FF0EE3CF1FF02E
:104930001200D9CFE6FFDACFE6FFE1CFD9FFE2CF11
:10494000DAFFFB0EDBCF00F0FC0EDBCF01F0000145
:10495000800E01141AE1FB0EDBCFE9FFFC0EDBCF6A
:10496000EAFFEECFF3FFEDCFF4FFEE2A000EEF22C9
:10497000F3CFE9FFF4CFEAFFFD0EDBCFEFFFEF50FF
:10498000016AF36E01C0F4FF10D0FB0EDB50FE088D
:1049900006E1FD0EDBCFE6FF62EC26F005D0FD0E52
:1049A000DBCFE6FF03EC00F0E552E552E5CFDAFF9E
:1049B000E7CFD9FF1200D9CFE6FFDACFE6FFE1CF8C
:1049C000D9FFE2CFDAFFFD0EDB50C96EC6AE02D0D2
:1049D000FF0E2BD00F0EC61408080FE00F0EC614E2
:1049E0000B080BE0C6889EA6FED7C750040B03E158
:1049F000C750010B17E0000E18D00F0EC6140808A0
:104A000004E00F0EC6140B0810E1C7B0FED7C75064
:104A1000040B01E0010E006E1F0EC5140010F7E13B
:104A2000C5AC02D0FE0E01D0000EE552E5CFDAFF94
:104A3000E7CFD9FF1200D9CFE6FFDACFE6FFE1CF0B
:104A4000D9FFE2CFDAFFAC6AAB6AFD0EDBB0AC880F
:104A5000DBA202D0AC8CAB8CDBB4AC8EDBA602D07C
:104A6000AB8801D0AB8ADBB8AC84DBBAAB86DBACFD
:104A700002D09D8A01D09D9ADBAE02D09D8801D0E4
:104A80009D98FB0EDB50AF6EFC0EDBCF01F001C03A
:104A900000F0016A0050B06EAC8AAB8EE552E5CFF3
:104AA000DAFFE7CFD9FF12001C502102F3CF18F034
:104AB000F4CF19F02202F3501926000EF4201A6EDA
:104AC0001C502302F3501A26000EF4201B6E1C50BB
:104AD0002402F3501B261D502102F3501926F450D6
:104AE0001A22000E1B221D502202F3501A26F450E7
:104AF0001B221D502302F3501B261E502102F3508F
:104B00001A26F4501B221E502202F3501B261F505F
:104B10002102F3501B2612001B6A1A6A196A186ACE
:104B2000200EE76ED8901C361D361E361F361836FE
:104B300019361A361B362150185C2250195823504A
:104B40001A5824501B5809E32150185E2250195A54
:104B500023501A5A24501B5A1C2AE72EE4D712005D
:104B6000D9CFE6FFDACFE6FFE1CFD9FFE2CFDAFF18
:104B7000E652F20E0F013717ABAC03D03791ABB052
:104B80003781ABB43785ABB23787AE50DF6EDF50BD
:104B9000E552E552E5CFDAFFE7CFD9FF1200D9CFD2
:104BA000E6FFDACFE6FFE1CFD9FFE2CFDAFFE65248
:104BB000E652FC0EDBCFDEFFDBCFDDFF010EDB506C
:104BC000CF6EDF50CE6EE552E552E552E5CFDAFF0B
:104BD000E7CFD9FF1200D9CFE6FFDACFE6FFE1CF6A
:104BE000D9FFE2CFDAFF3F0EC716C66AC56AFD0ECF
:104BF000DB50C612FC0EDB50C712C68AE552E5CF69
:104C0000DAFFE7CFD9FF1200FF0EE3502D6EEF0E53
:104C100001D0F30EE76EE72E0BEF26F00C0E2C6E94
:104C2000E76AE72E11EF26F02C2E10EF26F02D2E3E
:104C300009EF26F01200D9CFE6FFDACFE6FFE1CF89
:104C4000D9FFE2CFDAFFACAC04D0AC900F0137B3A0
:104C5000AC80FD0EDB50AD6EE552E5CFDAFFE7CF5D
:104C6000D9FF1200F36AF46AFF0EE124E96EFF0E29
:104C7000E220EA6EED6607D02F0EEF6404D03A0E04
:104C8000EF6001D0F32A1200380EF36E00EE00F050
:104C90000F0E01D81200EA6002D0EE6AFCD7F35082
:104CA000E9601200EE6AFCD71EEE00F02EEE00F076
:104CB000F86A279CB0EC23F0A2EC26F0B5EC0FF0DC
:104CC000FBD71200FF0EE350ACBA04D0AF6AAB8E34
:104CD000AC8A949CACA2FED7AD6EF36EF46A12005F
:104CE0001B6A080EE76ED8901F361B3624501B5CDB
:104CF00002E31B6E1F2AE72EF7D71200FF0EE350C8
:104D0000E84E1200000000D000D000D0E82EFAD704
:104D10001200C450036E026AC3500210F36E03C047
:104D2000F4FF1200303132333435363738396162AE
:104D30006364656600FFC250020B01E0010E1200C1
:104D4000C2821200120080250000C845EE450E46C2
:104D50003B464C4650466E468346C845EE450E4699
:104D60003B464C4650466E468346303030303030FD
:104D70003030003132333435363738393031323330
:104D80003435360080084A616E762E0046657672AC
:104D90002E004D6172732000417672696C004D6186
:104DA000692020004A75696E20004A75696C2E00E2
:104DB000416F75742000536570742E004F63746FDB
:104DC0002E004E6F76652E00446563652E004469A3
:104DD0006D616E004C756E6469004D6172646900AE
:104DE0004D65726372004A657564690056656E644C
:104DF000720053616D656400FFFFFFFFFFFFFFFF5F
:104E0000FFFFFFFFFFFFFFFFFFFFFFFFFFFFFFFFB2
:104E1000FFFFFFFFFFFFFFFFFFFFFFFFFFFFFFFFA2
:104E2000FFFFFFFFFFFFFFFFFFFFFFFFFFFFFFFF92
:104E3000FFFFFFFFFFFFFFFFFFFFFFFFFFFFFFFF82
:0200000400F00A
:1000000050726F6A65743A31384632364B3232205C
:1000100020554152543120425420200D0000000050
:1000200056657273696F6E2032302F30382F323040
:10003000313320202020202020202020200D0A00E5
:10004000506F727420436F6D206F757665727420E7
:100050002620496E69742048415244572E0D0A00EB
:10006000426F75636C6520656E2032205365632096
:1000700020203C4553433E2065786974200D0A00DA
:1000800041766563205541525431204841524457CE
:100090004152452E2E2E2E2E2E2E2E2E2E0D0A00A5
:1000A0007061756C666A756A6F40667265652E660A
:1000B0007220202020202020202020202020200D01
:1000C0004D504C4142204944452056382E3931206C
:1000D0002020202020202020202020202020200D33
:1000E0004331382076332E34352E303020202050C6
:1000F00069634B697433202020202020200D0A00E2
:10010000312E6D657373616765206F76657220317E
:100110003030682E2E2E2E2020202020230D0A0085
:10012000322E6D657373616765206F76657220315D
:100130003230682E2E2E2E20202020202A0D0A005C
:1001400020202020202020202020202020202020AF
:1001500020202020202020202020202020202000BF
:10016000FFFFFFFFFFFFFFFFFFFFFFFFFFFFFFFF9F
:10017000FFFFFFFFFFFFFFFFFFFFFFFFFFFFFFFF8F
:10018000FFFFFFFFFFFFFFFFFFFFFFFFFFFFFFFF7F
:10019000FFFFFFFFFFFFFFFFFFFFFFFFFFFFFFFF6F
:1001A000FFFFFFFFFFFFFFFFFFFFFFFFFFFFFFFF5F
:1001B000FFFFFFFFFFFFFFFFFFFFFFFFFFFFFFFF4F
:1001C000FFFFFFFFFFFFFFFFFFFFFFFFFFFFFFFF3F
:1001D000FFFFFFFFFFFFFFFFFFFFFFFFFFFFFFFF2F
:1001E000FFFFFFFFFFFFFFFFFFFFFFFFFFFFFFFF1F
:1001F000FFFFFFFFFFFFFFFFFFFFFFFFFFFFFFFF0F
:1002000020202020202020202020202020202020EE
:100210002020202031384632364B32325F42545F44
:1002200059435F4D43552E205254432D445331338F
:100230003037202B204C434420493243566572739B
:100240007573203133303832346220433138200026
:10025000496E69742055415254312039363030622C
:1002600064732020496E69742052544320445331F2
:100270003330372020202020496E6974206D6F6450
:10028000756C652059432D4D435520204E6F206CD1
:10029000696E6B20696620617070616972656420A7
:1002A00031384632364B32325F42545F59435F4DEC
:1002B0004355202031384632364B32325F42545F4C
:1002C00059435F4D4355202031384632364B323248
:1002D0005F42545F59435F4D43552020FFFFFFFFAE
:1002E000FFFFFFFFFFFFFFFFFFFFFFFFFFFFFFFF1E
:1002F000FFFFFFFFFFFFFFFFFFFFFFFFFFFFFFFF0E
:10030000FFFFFFFFFFFFFFFFFFFFFFFFFFFFFFFFFD
:10031000FFFFFFFFFFFFFFFFFFFFFFFFFFFFFFFFED
:10032000FFFFFFFFFFFFFFFFFFFFFFFFFFFFFFFFDD
:10033000FFFFFFFFFFFFFFFFFFFFFFFFFFFFFFFFCD
:10034000FFFFFFFFFFFFFFFFFFFFFFFFFFFFFFFFBD
:10035000FFFFFFFFFFFFFFFFFFFFFFFFFFFFFFFFAD
:10036000FFFFFFFFFFFFFFFFFFFFFFFFFFFFFFFF9D
:10037000FFFFFFFFFFFFFFFFFFFFFFFFFFFFFFFF8D
:10038000FFFFFFFFFFFFFFFFFFFFFFFFFFFFFFFF7D
:10039000FFFFFFFFFFFFFFFFFFFFFFFFFFFFFFFF6D
:1003A000FFFFFFFFFFFFFFFFFFFFFFFFFFFFFFFF5D
:1003B000FFFFFFFFFFFFFFFFFFFFFFFFFFFFFFFF4D
:1003C000FFFFFFFFFFFFFFFFFFFFFFFFFFFFFFFF3D
:1003D000FFFFFFFFFFFFFFFFFFFFFFFFFFFFFFFF2D
:1003E000FFFFFFFFFFFFFFFFFFFFFFFFFFFFFFFF1D
:1003F000FFFFFFFFFFFFFFFFFFFFFFFFFFFFFFFF0D
:020000040030CA
:0E0000000023193C009D84000FC00FE00F404C
:020000040020DA
:08000000FFFFFFFFFFFFFFFF00
:00000001FF
